:102B9E0033302E3120202020000000420D00204333
:102BAE000D0100440D0120450D0010460D0030476B
:102BBE000D0110480D0130490D00084A0D00284B3B
:102BCE000D01084C0D01284D0D00184E0D00384F0B
:102BDE000D0118500D0138510D0200520D0208530F
:102BEE000D0210540D0218550D0220560D022857D5
:0D2BFE001201025F0D02610002630C02650E
:0F2F6800C120C128C1254202020000C121C1229F
:10149A00900347E0FCA3E0F5828C83E49325E022E5
:1014AA00246AF582E43402F583EEF0A3EFF0229089
:1014BA0003541210F79003541210CBC374FF9BFF0E
:1014CA0074FF9AFEE499FDE498FC9003541210F715
:1014DA0090035422E0FFC374FF9FFD900349E0FB91
:1014EA00900347E0FFA3E090034DCFF0A3EFF02273
:1014FA009390026E75F0FFA4FFE5F0F0A3EFF022DF
:10150A00FFE49400FE745B2FF582740C3EF583E4CD
:10151A00227C007DFF120ECBEE90034FF0A3EFF07A
:10152A0022900354121160900005120E6AFF900077
:10153A0006120E6AFD900004020E6A900343E0FF51
:10154A00C374FF9FFF22E0FEA3E0F5828E8374013D
:10155A0093FE740293FFF5828E83E0FCA3E0FD22E2
:10156A007B017A03794190035412116090000312AF
:10157A000E6AFF90029BE06F22AC58AD597A007B4D
:10158A0001EDAE0422120EDD90035CEEF0A3EFF043
:10159A00C322900C5B9375F0FFA4FF222470F5829E
:1015AA00E43402222476F582E4340222247CF58291
:1015BA00E4340222FFE0FE2FFFC39E22E0FEA3E0F6
:1015CA00FFA3E0FDA3E0FBA3E02285178285168333
:1015DA0022E542F0A3E546F0AB5EAD5A22E543F0C0
:1015EA00A3E547F0AB5FAD5B22E544F0A3E548F025
:1015FA00AB60AD5C22E545F0A3E549F0AB61AD5DBA
:10160A00227E007C00020ECB3EF583E4F0A322E4A6
:10161A007BFFFAF9F8021004C374FF9DF0A374FF6C
:02162A00F022AC
:0B32AF00EEF0A3EFF0A3EDF0A3EBF0B6
:0432BA00A281B32218
:0C32E7007B017A027905900267021160F9
:101B97007B017A03794112306AEF7003021CB5901A
:101BA7000343E01211691C12041C23051BDC141BE0
:101BB700CC161BD0171BE11A1BFB1B1C061D1C0C8C
:101BC7001E00001C3DD2248002C224A224922812A7
:101BD70025B2021C3DD220021C3D7B017A037941CC
:101BE700900351121160120E51FE90029BE0FF6E9E
:101BF7007044800590029BE0FF12324A021C3D129E
:101C07003364021C3D123377021C3D12156A70269D
:101C170030241B12152BFB122C0B801212156A7025
:101C27001530240A12152BFB122955121CE39002BA
:101C37009BE0FF123219202403021B97900343E015
:101C470014601B24FA602314604A24066003021BF5
:101C570097121CB690037DF012337D021CAF121C45
:101C6700B690037DF0121CE3803E121CCC12153F88
:101C7700FD900005120E6AFBC00390035712114036
:101C8700900006120E6A90035DF0D00312285712D7
:101C97001CED8014121CCC12153FFD900005120E8E
:0E1CA7006AFB1224E5121CED12331E021B977D
:101CB5002212328E7B017A03794190035112116011
:101CC500900003120E6A2212328E7B017A0379414B
:101CD500900357121160900003120E6AFF22123012
:101CE500AE1230251225B2221230AE123025122541
:021CF500B22219
:1011E8001231631232E7E5A0F515750B071231E6E7
:1011F800123002D2AF90029B7423F0FF1232DA430E
:10120800F601123344E490037DF01230AE1225B299
:10121800E51260FCE51260FCE51260FCE490034016
:10122800F0900340E0F9C36480948440030212D232
:10123800E0FF244AF8E6FDEF3395E0FEEF25E0FFF6
:10124800EE33FE74242FF5827403121612EDF0901B
:101258000340E0FD244AF8E6FCEDFB3395E0FA7420
:10126800062BF58274033AF583ECF0745429F8E6FA
:10127800FD74382FF5827403121612EDF0FFE9FDA4
:101288003395E0FC74102DF58274033CF583EFF080
:10129800744E29F8E6FBED25E0FFEC33FE742C2FA5
:1012A800F5827403121612EBF0744E29F8E6FFE982
:1012B800FD3395E0FC740A2DF58274033CF583EF49
:1012C800F0900340E004F00212291232BA90029A18
:1012D8005005740AF080037432F030212490020221
:1012E80074FFF5F0120F32900202E07002A3E07072
:1012F80010C22190029BE0FF7BFF7A2B799E122C73
:10130800DE121CF730250A90029BE0FF123200C261
:101318002530220FE490037DF012337DC228122578
:10132800B2C222E4F512302303021407900340F0FE
:10133800900340E0FF2408121491FE2404FFEE24D9
:101348000C121491FE2408FFEE2412FD1217B0901F
:101358000340E004F0E0C36480948440D330290360
:101368001225B2302604C226D227AE58E559780590
:10137800CEC313CE13D8F954037E2B7FFF600B9096
:1013880003451215DB121E4980099003451215DB2F
:1013980012192FAE58E5597807CEC313CE13D8F9D2
:1013A80054037E2C7F02600B9003451215E7121E32
:1013B8004980099003451215E712192FE558C31300
:1013C80054037E2C7F05600B9003451215F3121E03
:1013D8004980099003451215F312192FE558131384
:1013E8001354037E2C7F08600B9003451215FF12DF
:1013F8001E4980099003451215FF12192FC22712A2
:1014080032BA5035C374FF956212150A1214FAC322
:1014180074FF956312150A939002741214FEC37434
:10142800FF956412150A12159F90027A121503C3CC
:1014380074FF956512150A8023E562900C5B1214FF
:10144800FAE56312159C900274121503E5641215EF
:101458009C90027A121503E565900C5B12159F901B
:101468000280121503122E3F122F3D780E74FF12C0
:1014780010D9EC4D4E4F700B7511A0751086750F75
:0914880001F50E121B970212E29D
:09149100FD1217B0900340E022A7
:10327800758850758922758E0C758AAE758CAE75F9
:063288008BC7758DC72203
:10316300E4F5D975FF8075EF0212333212330A1278
:0B317300304812329F12333B023278CA
:09333200E4F5B1F5A975B283229E
:1030480075A4CF75D40875F2F875A5F875A71F751E
:10305800B0FF75A0FF7590FF7580FF75E10675E2FA
:02306800402204
:10329F0075BCFC75E8C075BA1F75D10843E60822E6
:09333B0043E61075D983D2DE22AD
:0A330A0075A14075F801E4F5A22258
:101CF700E5097003021E481211691D1A021D6204CC
:101D07001D93081DB7101DDB201E0C401E218000EF
:101D1700001E3FAC58AD59EDAE047803CEC313CEC9
:101D270013D8F9FFED54E7FDEF2401FF7A00EF54D4
:101D370003FB7E007803C333CE33CED8F9FFEE4CD6
:101D4700F558EF4DF559EB64034A6003021E3F85D2
:101D57005858E55954E7F559021E3FAE58AF59ACEC
:101D670006EF54FCFDEF2401FFE43E7E00EF540331
:101D7700FFECF558EF4DF559EF64036003021E3F82
:101D8700855858E55954FCF559021E3F12158378BA
:101D970002CEC313CE13D8F95401FFED54FBFDEF68
:101DA7006B7E0054017802C333CE33CED8F9804A14
:101DB7001215837805CEC313CE13D8F95403FFED5C
:101DC700549FFDEF6B7E0054037805C333CE33CEAB
:101DD700D8F980261215837807CEC313CE13D8F906
:101DE7005403FFEC54FEFCED547FFDEF6B7E005473
:101DF700037807C333CE33CED8F9FFEC4EF558ED51
:101E07004FF5598033AC58ECC3135403FFEC54F926
:101E1700FCEF6401540325E08017AC58EC1313134F
:101E27005403FFEC54E7FCEF64015403333333549A
:101E3700F84CF558E559F559E4F5091225B2123170
:021E47000E2269
:10312B007E80E4FDEE5F6004D2878002C287C28698
:0B313B00EEC313FED2860DEDB408E9D0
:013146002266
:1025B200E4FDC2293005010D300604ED4402FDE5BB
:1025C20059540314600D14601024027010ED44106D
:1025D200FD800AED4420FD8004ED4440FD302804D6
:1025E200ED4480FDAF0512312BE4FDAE58E559787C
:1025F20005CEC313CE13D8F954036004ED4401FD94
:10260200AE58E5597807CEC313CE13D8F9540360F8
:1026120004ED4402FDE558C31354036004ED440481
:10262200FDE55813131354036004ED4408FDAF0590
:1026320012312BC2AF530B3FAE58E5597803CEC3CC
:1026420013CE13D8F9540314600C14600E240270D4
:102652000D430B408008430B808003430BC0850B66
:1026620090D2AFAE58E5597802CEC313CE13D8F943
:032672001392B40C
:012675002242
:031A2400021F8A14
:101F8A00C0E0C083C082C0D075D000C000C005C008
:031F9A0006C00777
:101F9D0020DF0302209BE5A05401FF70027F03E5C3
:101FAD00A0F5086515600CE5086515F50C751403AD
:101FBD00850815E51470030220801514E5146003DF
:101FCD00022080E50820E01330200E9002027407F5
:101FDD00F0A374D0F0D2218002D222E508B4FF0321
:101FED00750A00E50C30E025E50830E020E50AF43F
:101FFD00601BC221900202E07002A3E0600F30204E
:10200D000CA224B39224A22492281225B2E50C30FE
:10201D00E10DE50830E108E50AF46003750902E514
:10202D000C30E208E50820E203750904E50C30E305
:10203D0008E50820E303750908E50C30E408E50818
:10204D0020E403750910E50C30E508E50820E503EB
:10205D00750920E50C30E608E50820E60375094012
:10206D00E50C30E708E50820E703750980E5096010
:10207D0002F50AC2DFE54145406013E541154170A7
:0E208D000215401445407006C205C206D22955
:10209B00D007D006D005D000D0D0D082D083D0E0EE
:0120AB003202
:103232001215D4E493F5BB530BC71215D474019342
:08324200420B850B90D2EC2237
:0933440075162B7517A702323231
:031A2100022ABDD9
:102ABD00C0E0C083C082C0D075D000C000C001C0CE
:102ACD0002C003C2ED1215D4740293F8A6BE1215FE
:102ADD00D4740393F8760174042517F517E43516AD
:102AED00F516FAA9177BFF74FF902BFFF47009E51B
:102AFD001765827003EA6583701475162B7517A719
:102B0D0090029AE00513B51305D226751300123203
:102B1D0032D003D002D001D000D0D0D082D083D01B
:022B2D00E03294
:061A1B00E5A120E7FB221B
:08334D00E5A120E7FB8FA3229C
:102E3F007D6A7C027B30C283E4FAE4FF12334DAF2C
:102E4F000312334D8D828C83E0FF12334DA3E0FFCD
:102E5F0012334D74022DFDE43CFC0AEAB403DB127D
:092E6F001A1BD2830BEBB438CD21
:012E78002237
:1022DE00900347EEF0A3EFF090034AEBF090034922
:0222EE00EDF011
:1022F000D394F0400E90034BE0FF900349F074FF3D
:102300009F804F900349E0FFC3944C500AE4F09043
:10231000034D74FFF0803FEFC394B3900349400630
:1023200074FFF0E4802CE0FFE412152390034F7457
:10233000FF75F0B4120F3290034FE0FEA3E0FF12DE
:10234000151B7D67120EDD121522900349F0C37430
:10235000FF9F90034DF090034AE0FFD394F04013A9
:1023600090034CE0FE74FF9E90034AF090034EEE03
:10237000F0802DEFD3944C90034A400674FFF0E4B4
:10238000801AE0FF7E0012152212151B7D4C120EE2
:10239000DD12152290034AF0C374FF9F90034EF0A4
:1023A00090034DE0FF90034AE0FD1232BE12149AF2
:1023B0001214AA9003491223E812149A1215A612B5
:1023C00014B190034D1223E812149A1215AE121490
:1023D000B1900349E0FF90034EE0FD1232BE1214AB
:0723E0009A1215B61214B1A8
:0A23E70022E0FFA3E0FD1232BE2247
:052A4900900353EBF0C7
:102A4E001232BE900353E0900C5B93FD7C0012118A
:102A5E008F1216191214B91210BF78051210ACE4A9
:102A6E007B03FAF9F8120F799003581214D712104B
:102A7E00BF9003581210CB120F6B1214D41210CB3E
:102A8E00C000C001C002C003900353E0FFE4FCFD90
:102A9E00FE9003581210CB120F79121619D003D0D4
:0E2AAE0002D001D000120F5E1214B91210BF38
:012ABC0022F7
:052F910090034CEBF081
:102F9600122EE390034EE02FFF90034DE03EFE908D
:102FA600034CE090095B93FD122EFF7DFF122EFF6E
:012FB60022F8
:102C7600EFC3941950107DB412160B7D1912158FDF
:102C860074FF9FFB804FEFC3944050107D2F1216A8
:102C96000B7D2712158F74689FFB8039EFC3947FD5
:102CA600501D7E007C007D07120ECBEF7805CEC34B
:102CB60013CE13D8F9FF121592742A9FFB8016EFD4
:102CC60075F007A4AEF07806CEC313CE13D8F9FF7D
:072CD600C3741C9FFBAF0358
:012CDD0022D4
:0E32BE007BFF122EE3EEFF122C76EF7F00FE58
:0132CC0022DF
:10192F009003411232AF50159003411215C6900328
:10193F004BF0900346E090034CF00222DE900343FD
:10194F00E0FFD394F04006900345E0801DEFC39471
:10195F004C5003E48014900343E0FFC394B340055D
:10196F0074FFF08009EF9008A893900343F0900361
:10197F0044E0FFD394F04006900346E08013EFD38A
:10198F00944C900344400574FFF08009E09008A741
:10199F0093900344F01215451219F312149D12146B
:1019AF00AA900343E0FF1219F312149D1215A61209
:1019BF0014B11215451219E212149D1215AE12141C
:1019CF00B1900343E0FF1219E212149D1215B612E3
:1019DF0014B122A3E0FEC374FF9EFD7BFF122EE322
:1019EF0090034122A3E0FD7BFF122EE390034122DF
:10162C0090034AEEF0A3EFF090034DEBF090034CD7
:02163C00EDF0CF
:10163E00C374FF9DF020270302179B90034EE0908A
:10164E00034C1215BE500574FFF0800590034CEF4D
:10165E00F090034FE090034D1215BE500574FFF04D
:10166E00800590034DEFF090034A12155090034CF5
:10167E00E0F9C3947F50388F828E83C083C082E09E
:10168E00FAA3E0FBE9FFC3747F9FFFE49400FEEF33
:10169E007803CEC313CE13D8F92401FFE43EFEC364
:1016AE00EB9FFFEA9ED082D083F0A3EFF0803AE961
:1016BE00D3947F4034E92481FFE434FFFEEF7803B6
:1016CE00CEC313CE13D8F92401FFE43EFE90034A95
:1016DE00E0FAA3E0F5828A83740193FA740293F51B
:1016EE00828A83EE8FF0120F3290034DE0900352F8
:1016FE00F0EC540314601414601C14602124037065
:10170E0028ED90034CF0E4A3F0801E90034C74FF80
:10171E00F0EDA3F0801390034C121622800BE49090
:10172E00034CF0C374FF9DA3F0900352E0FB12151F
:10173E0049EF900350F0A3E4F090034C121548A328
:10174E00E0FD122A4990034A12149D1214AA900326
:10175E004CE0FFA3E0FD900352E0FB122A499003F8
:10176E004A12149D1215A61214B190034C1215486C
:10177E0012179C12149D1215AE1214B190034CE068
:0D178E00FF12179C12149D1215B61214B113
:10179B0022A3E0FEC374FF9EFD900352E0FB122ACE
:0517AB004990034A22F1
:031E4900900341C2
:101E4C001232AF50159003411215C690034EF0900C
:101E5C000346E090034FF002162C202703021F7D4F
:101E6C00900345E0FF9003431215BF500574FFF03B
:101E7C008005900343EFF0900346E0FF900344127B
:101E8C0015BF500574FFF08005900344EFF09003EC
:101E9C00411215508F828E83C083C082E0FEA3E076
:101EAC00FF900343E075F002900A5B121134E49347
:101EBC00FA740193FBC3EF9BFFEE9AD082D083F0B0
:101ECC00A3EFF0900344E0900349F0EC540314604A
:101EDC001414601C14602124037028ED900343F04B
:101EEC00E4A3F0801E90034374FFF0EDA3F0801385
:101EFC00900343121622800BE4900343F0C374FF4B
:101F0C009DA3F0900349E0FB121549EF900347F0B5
:101F1C00A3E4F0900343121548C007A3E0FD12148C
:101F2C00EAD007122F9190034112149D1214AA901B
:101F3C000344E01214E4121F7E12149D1215A61213
:101F4C0014B1900343121548C007A31214DED00736
:101F5C00122F9190034112149D1215AE1214B190D0
:101F6C0003441214DE121F7E12149D1215B61214A5
:011F7C00B1B3
:0D1F7D0022900343E0FF122F9190034122B8
:102F3D00E553D394C04007D2B1C2B2C2B322C2B1DD
:102F4D00E553D394404005D2B2C2B322C2B2E55389
:0B2F5D00D394204003D2B322C2B32261
:1030EF00E475F001120F4885F082F5832275B7A5BC
:0F30FF0075B7F18F828E8322EEF0A3EFF0A3223C
:10317E00A2AFE433FCC2AF758F011230FCEDF0E468
:09318E00F58FAF04EF24FF92AFAE
:013197002215
:1019FF00A2AFE433FDC2AF758F031230FCE4F0F5F4
:081A0F008FAF05EF24FF92AF39
:011A170022AC
:102DBF0090036F123107ECF0A3EDF0EB4A60319006
:102DCF00036FE0FEA3E0FFA3E0FCA3E0F5828C839A
:102DDF00E0FD12317EEB1B70011A900371E475F068
:102DEF0001120F3290036FE475F001120F3280CB96
:012DFF0022B1
:08335500E4900000F0A3F02257
:102FB700900000E0FEA3E0FF1219FF900000E0FE82
:102FC700A3E0FF7C007D027B007A02122DBFE49014
:062FD7000000F0A3F0224F
:0A29D200A905900369EEF0A3EFF0F1
:1029DC00EE54FEFE900000E0FCA3E0FD7002EE6CF5
:1029EC006042ED4C6003122FB7900369E0FEEE5489
:1029FC00FEFE7F00900000F0A3EFF090036B12310D
:102A0C00077400F0A37402F07E0290036B1230EF97
:102A1C00E493FD90036D1230EFEDF0EF1F70011E8B
:102A2C00EF4E70E6900369E0FCA3E0FDEC5401FC72
:0C2A3C0074022DF58274003CF583E9F073
:012A4800226B
:102E790090036212310712116090036774FFF5F035
:102E8900120F4845F06020900362E475F001120FBB
:102E990048AFF0FE900364E475F001121149120E77
:082EA90051FD1229D280D22252
:102F77004202FC00004202A700004202A20000C178
:052F87002CC12BC12A42
:102D360090029DE475F001020F32D39002FDE094FB
:102D4600009002FCE06480948022E0FEA3E024A9C7
:102D5600F5827402229002A2F0A3F02274FFF5F02D
:102D6600020F32E0F5C2C2C5C2C49002E922FCE5F8
:052D7600F064404C2256
:0A331400C22BC22CE49002A6F022A6
:1030CF00E49002FCF0A3F09002A7F0A3F0A3F0129B
:1030DF002D5B90029DF0A37440F0E49002A5F022C6
:06336B001233140230CF02
:0D32CD0075C19043E6019002A47401F02247
:10328E0043C140E5C120E5FB12336BE49002A4F08C
:01329E00220D
:0A331E0053C1BF9002A47401F02215
:0D32DA00AE071232CD9002A1EEF002336B70
:102FDD00E490036BF0A3F0302B02FF22202CFDD2E6
:102FED002B90029FE4F0A37410F09002EAEFF0E44E
:042FFD00A3F07F01BD
:0130010022AC
:102F1100302B0A90029FE07002A3E070037F002231
:102F210090029F122D629002EBE0FE04F074EC2EF1
:0C2F3100F582E43402F583EFF07F01220A
:0B32FF00302B07C22BD22C12332822E8
:0A332800E5C120E5FBC2C4D2C522B6
:102B2F009003651211609002A4E07002FF229003DF
:102B3F0068E0FE6005D3941040037F0022122FDD62
:032B4F00EF6049EB
:102B5200E490036AF0900368E0FF90036AE0FEC32A
:102B62009F501F9003651211408E82758300120ED2
:102B72006AFF122F11EF7002FF2290036AE004F045
:102B820080D3E49002A6F01232FF900369E0700352
:092B9200202CFD9002A6E0FF22B8
:032B9B007FFF2297
:0B27320090035D121160900360EDF059
:10273D00E4FF122D4050012253E6FE9002A2122D0D
:10274D00503EF583E0FF9002A2122D39122D7470C8
:10275D0003122D5B122D36E4FE900360E0FDEEC3F7
:10276D009D5035EEC39F50309002A2E0FC122D52C9
:10277D003CF583E0FD90035D1211408E8275830060
:10278D00ED120EA99002A2122D39122D74700312A2
:10279D002D5B122D360E80C1EEC39F50149002A2F8
:1027AD00122D39122D747003122D5B122D360E80E1
:1027BD00E79002FC122D6243E601900360E0FEEF0C
:0827CD00C39E50028002AF061A
:0127D50022E1
:0C32F300122D4040047F0180027F002269
:031A1800021A2788
:101A2700C0E0C0F0C083C082C0D075D000C000C085
:031A370006C007DF
:101A3A00C22FE5C054FE1211691B06081B060A1ABA
:101A4A00CF0C1ACF0E1B64101B64121AD5221AE08F
:101A5A00281AE02A1AD52C1AD52E1AC2C01A82C2FE
:101A6A001A74E01A74E200001B6FC22A9002EA128A
:101A7A002D6974FFF0021B719002E9E0FFB4FF0BBD
:101A8A009002EB122D69E4F0021B719002EBE0FE6A
:101A9A00EFC39E50179002E9E0FF04F074EC2FF5B3
:101AAA0082E43402F583E0F5C2021B71D2C49002CB
:101ABA00A6E4F0C22C021B719002A674FDF0D2C5F6
:101ACA00C2C4021B719002E974FFF0D22AC2C4C2D6
:101ADA00C1D2C5021B71E5C260079002A1E0B5C27E
:101AEA000E90029CE4F0C2C5C2C4D2C1021B71C2EC
:101AFA00C4C2C1302A028067C2C5806B90029CE0D2
:101B0A007020E5C2F0E0FFC390029EE09F7480F867
:101B1A0090029DE064809850031230CF90029CE0BE
:101B2A0004F090029D122D629002A7122D503EF5EC
:101B3A0083E5C2F09002A7122D39FEE5F064404E0B
:101B4A0070069002A7F0A3F090029CE014F07006D1
:101B5A009002FC122D3AD2C1800DC2C4302A08C2AA
:101B6A002AD2C58002D22F302F1053C17F43C180A1
:0C1B7A00C2C5C2C4C2C1C22FC22CC2C06E
:101B8600D007D006D000D0D0D082D083D0F0D0E01D
:011B9600321C
:05337100E5C15420FF3E
:013376002234
:103198007B01E4900362F0227422F0A3EFF0A322F3
:0A31A8007B01E4900362F07D042235
:0B2E000090035E121160900361EDF082
:102E0B00E4900363F090035E121140900361E09035
:102E1B000368F0900362E0900369F0E4FF122B2F3C
:102E2B00EFB4FF0D900363E0FE04F0EEC394034098
:032E3B00D47E0042
:012E3E002271
:06306A0090035A121160F0
:103070007E007F007D101211BC90035A1211407D1A
:0B30800010122732EF7002FF227F01C8
:01308B002222
:102CDE009003411231A07413F0120E51900344F080
:102CEE00900001120E6A900345F0900002120E6AD7
:102CFE00900346F0900003120E6A900347F0900086
:102D0E0004120E6A900348F0900005120E6A9003AA
:102D1E0049F0900006120E6A90034AF07A03794148
:082D2E001231987D0A022E000B
:103200009003411231A07403F0A374FFF07A0379A4
:09321000411231987D04022E00E8
:10324A0090035A1231A0741CF0A374FFF07A037928
:07325A005A1231A8022E00F8
:10321900E490035AF0A3EFF0A3740AF0A3EFF07A55
:0932290003795A1231A8022E00AB
:102EB10074FFF5F0020F32EFF0A3ECF0A3EDF0A3F5
:102EC100021160D2C1C2C4D2C5E4FF90038EF022C8
:102ED100E5188519F0020F32E025E044A0F5C27F24
:022EE1000322CA
:07335D0043C14053E6FE22CC
:0623F100900372122EB8E9
:1023F70090037B7403F0A374E8F0E5C120E5FB12BA
:102407002EC430C0FDE5C054FEFE244070030224F4
:102417009724FE601A24E2600924FE600524E20284
:10242700249FC2C5EF7077900372122ED9806FEF89
:10243700B4030A900373E0F5C27F058061EFB4052A
:102447000B900373A3E0F5C27F068052EF6406701A
:102457002D90037AE0900375700875F00112114909
:102467008003121140120E51F5C2900378122EB15B
:10247700900378E07002A3E070247F078020EFB418
:102487000706D2C47F09801690038E7405F0800E6C
:1024970090038E7402F0800690038E7401F0EFB4FF
:1024A7000904C2C0803290038EE0FE6406600EEE1F
:1024B700B4021290037B122EB145F06008D2C5E436
:1024C70090038EF0FF90038EE06008C2C5D2C4C2AD
:0D24D700C08005C2C0022409E5C120E5FB5C
:0124E40022D5
:0620AC0090036A122EB839
:1020B2009003727403F0A374E8F0E5C120E5FB120B
:1020C2002EC430C0FDE5C054FEFE12116920E800A6
:1020D20021713821468A2179C0210FC220EBE020EC
:1020E200EBE2000020E8022181C2C5EF70099003F3
:1020F2006A122ED9022187EF6401600302218790C0
:10210200036AE025E044A1F5C27F048078EFB403BE
:102112000A90036BE0F5C27F05806AEFB4050B906D
:10212200036BA3E0F5C27F06805BEFB40606D2C55F
:102132007F018051EFB404047F02804990038E74C2
:1021420005F0804190036DE475F001121149E5C27A
:10215200120E97900370122EB1900370E07002A3DA
:10216200E070087F09C2C1D2C4801A7F0280169033
:10217200038E7406F0800E90038E7402F080069037
:10218200038E7401F0EFB40904C2C0803290038E52
:10219200E0FE6406600EEEB40212900372122EB1DB
:1021A20045F06008D2C5E490038EF0FF90038EE004
:1021B2006008C2C5D2C4C2C08005C2C00220C4E544
:0421C200C120E5FB58
:0121C60022F6
:1021C700900369EFF090036C12116090036AECF0D2
:0321D700A3EDF085
:1021DA00751A00543FF51B543F604BC37440951B5E
:1021EA00FFE4951AFE90036FE0FCA3E0FDC39FECA9
:1021FA009E50068C188D1980048E188F191222B5DC
:10220A0060037F022290036A122ED1900371E0705C
:10221A000690036D122ED1C3900370E09519F090C9
:10222A00036FE09518F090036FE0F518A3E0F51935
:10223A00D3E5199400E5189400406DE5199440E53A
:10224A00189400500F1222B560037F0222E4F51899
:10225A00F51980DC900369E0FFA3E0FCA3E0FDA38D
:10226A00121140900378E4F0A37440F0900371E0F7
:10227A0090037AF01223F190038EE060037F02222A
:10228A0074C02519F51974FF3518F51890036AE416
:10229A0075F040120F32900371E0709490036D75DF
:0A22AA00F040120F3202223A7F00CA
:1022B40022900369E0FFA3E0FCA3E0FDA312114018
:1022C400900378E518F0A3E519F0900371E090030A
:0A22D4007AF01223F190038EE0224D
:10326100900370E4F0A304F01220AC90038EE060B0
:07327100037F01227F002210
:1031B20090038DEBF07B017A03798D90036FE4F03D
:0A31C200A304F0E4A3F01221C722D9
:10308C00C007900368E0FFA3E0900370CFF0A3EFBC
:10309C00F0D0071220AC90038EE060037F01227FFA
:0230AC00002200
:1031CC00C007900367E0FFA3E090036FCFF0A3EF7D
:0A31DC00F0E4A3F0D0071221C7228F
:1008A7000003070A0D1114171B1E2225282C2F32AF
:1008B70036393C4043464A4D5154575B5E61656843
:1008C7006B6F7275797C8083868A8D9094979A9ED8
:1008D700A1A4A8ABAEB2B5B9BCBFC3C6C9CDD0D36E
:1008E700D7DADDE1E4E8EBEEF2F5F8FCFF0003050B
:1008F700080A0D0F121417191C1E212326282B2D49
:10090700303235373A3C3F414446494B4E505355B8
:10091700585A5D5F626467696C6E717376787B7D28
:10092700808285878A8C8F919496999B9EA0A3A598
:10093700A8AAADAFB2B4B7B9BCBEC1C3C6C8CBCD08
:10094700D0D2D5D7DADCDFE1E4E6E9EBEEF0F3F578
:10095700F8FAFDFF4D4D4E4F4F50515152535454DD
:10096700555656575858595A5B5B5C5D5D5E5F5FDD
:1009770060616262636464656666676869696A6B19
:100987006B6C6D6D6E6F7070717272737474757657
:1009970077777879797A7B7B7C7D7E7E7F80808193
:1009A7008282838485858687878889898A8B8C8CD0
:1009B7008D8E8E8F9090919293939495959697970D
:1009C70098999A9A9B9C9C9D9E9E9FA0A1A1A2A349
:1009D700A3A4A5A5A6A7A8A8A9AAAAABACACADAE87
:1009E700AFAFB0B1B1B2B3B3B4B5B6B6B7B8B8B9C3
:1009F700BABABBBCBDBDBEBFBFC0C1C1C2C3C4C400
:100A0700C5C6C6C7C8C8C9CACBCBCCCDCDCECFCF3C
:100A1700D0D1D2D2D3D4D4D5D6D6D7D8D9D9DADB78
:100A2700DBDCDDDDDEDFE0E0E1E2E2E3E4E4E5E6B6
:100A3700E7E7E8E9E9EAEBEBECEDEEEEEFF0F0F1F2
:100A4700F2F2F3F4F5F5F6F7F7F8F9F9FAFBFCFC2F
:100A5700FDFEFEFFFF82FF83FF84FF85FF86FF8782
:100A6700FF88FF89FF8AFF8BFF8CFF8DFF8EFF8F2B
:100A7700FF90FF91FF92FF93FF94FF95FF96FF97DB
:100A8700FF98FF99FF9AFF9BFF9CFF9DFF9EFF9F8B
:100A9700FFA0FFA1FFA2FFA3FFA4FFA5FFA6FFA73B
:100AA700FFA8FFA9FFAAFFABFFACFFADFFAEFFAFEB
:100AB700FFB0FFB1FFB2FFB3FFB4FFB5FFB6FFB79B
:100AC700FFB8FFB9FFBAFFBBFFBCFFBDFFBEFFBF4B
:100AD700FFC0FFC1FFC2FFC3FFC4FFC5FFC6FFC7FB
:100AE700FFC8FFC9FFCAFFCBFFCCFFCDFFCEFFCFAB
:100AF700FFD0FFD1FFD2FFD3FFD4FFD5FFD6FFD75B
:100B0700FFD8FFD9FFDAFFDBFFDCFFDDFFDEFFDF0A
:100B1700FFE0FFE1FFE2FFE3FFE4FFE5FFE6FFE7BA
:100B2700FFE8FFE9FFEAFFEBFFECFFEDFFEEFFEF6A
:100B3700FFF0FFF1FFF2FFF3FFF4FFF5FFF6FFF71A
:100B4700FFF8FFF9FFFAFFFBFFFCFFFDFFFEFFFFCA
:100B57000000000100020003000400050006000772
:100B670000080009000A000B000C000D000E000F22
:100B770000100011001200130014001500160017D2
:100B870000180019001A001B001C001D001E001F82
:100B97000020002100220023002400250026002732
:100BA70000280029002A002B002C002D002E002FE2
:100BB7000030003100320033003400350036003792
:100BC70000380039003A003B003C003D003E003F42
:100BD70000400041004200430044004500460047F2
:100BE70000480049004A004B004C004D004E004FA2
:100BF7000050005100520053005400550056005752
:100C070000580059005A005B005C005D005E005F01
:100C170000600061006200630064006500660067B1
:100C270000680069006A006B006C006D006E006F61
:100C37000070007100720073007400750076007711
:100C470000780079007A007B007C007D007E007FC1
:100C57000080008100000000000101010101010185
:100C6700010101020202020202020202030303035C
:100C7700030303030304040404040404040505052F
:100C870005050505060606060606060707070707FC
:100C9700070708080808080809090909090A0A0AC4
:100CA7000A0A0A0B0B0B0B0B0C0C0C0C0C0D0D0D85
:100CB7000D0E0E0E0E0F0F0F0F1010101011111139
:100CC70012121212131313141414151515161617DE
:100CD700171718181919191A1A1B1B1C1C1D1D1E6A
:100CE7001E1F1F20202121222223242425262627D8
:100CF7002828292A2A2B2C2D2D2E2F303132333319
:100D07003435363738393A3B3C3E3F40414243451C
:100D17004647494A4B4D4E505153545657595B5CC1
:100D27005E6062646667696B6E70727476797B7DEC
:100D3700808285878A8D909295989B9EA1A5A8AB66
:100D4700AFB2B6B9BDC1C5C9CDD1D5D9DEE2E7EBE2
:040D5700F0F5FAFFBA
:1028D700900342E025E02414F582E43403F58322D3
:1028E700E47F01FEFDFC1210CBC3021096F8E6FB55
:1028F700C374FF9BFFE49400FEE49400FDE494009E
:10290700FC221210CB122D7B9003491210F7900373
:1029170042E0244222FEFDFC9003451210CBD30275
:102927001096120F6B9003451210F7E422900341A3
:10293700E0245A229003491210CB020F79E47BFF5F
:0E294700FAF9F822900342E0FF2442F8E6225B
:10300200D21ED21DD21CD21AD210D20FD20ED20D83
:10301200D20CD20BD20AD209D208D207C205C206FA
:03302200D229228E
:10302500C21EC21DC21CC21AC210C20FC20EC20DE0
:10303500C20CC20BC20AC209C208C207C205C20637
:03304500D229226B
:0817B000900341EFF0A3EDF0FE
:1017B8001228DBE0FEA3E0FFE4FCFDC004A905AAB3
:1017C80006AB07122915F8E6FFE4FED00012292916
:1017D800900343F0A3F07F02FEFDFCA31228ED4026
:1017E80008900343E4F0A304F074FF7FFE12291C61
:1017F800500874FF900343F0A3F0900343E0FEA366
:10180800E0FF4E700302192EEFF47002EEF4705AE6
:101818001228D7E0FEA3E0FFE4FCFD90035112106C
:10182800F79003511228E7500A9003511211030050
:10183800000001122934F8E6FFE4FCFDFE7BFFFA04
:10184800F9F8120F79900351122909F8E6FFE4FC20
:10185800FDFE12293B90034D1210F7122944900304
:071868004D1210BF122D7B91
:0F186F000218D7900343E07004A3E06401705F98
:10187E001229341228F4122944120F7990034912B6
:10188E0010F71228D7E0FEA3E0FBC374FF9BFFE422
:10189E009E1228FF90034D1210F790034D1228E769
:1018AE00500A90034D1211030000000190034912DB
:1018BE0010BF90034D1229091228F412293B122948
:0F18CE0044122D7BC374FF9FFF122934F8A60725
:1018DD0012294BFDEF1228DBE4F0A3EDF0FBE4FA47
:1018ED00F9F8900342E024FEF582E43402F583E03A
:1018FD00FFE4FCFDFE1229297F0512291C500F74EF
:10190D00FF7FFBFEFDFC9003451228ED50131231B5
:10191D000E12294BFE74FE2FF582E43402F583EE90
:01192D00F0C9
:01192E002296
:042F8C0041038C0071
:1027D60090035FE075F00E903A01121134AF82AEAD
:1027E6008322E475F001120F32900361E475F00163
:1027F600020F327B007A007958900367E4F0A374E5
:102806000EF02290035BEEF0A3EFF0E4900361F08C
:10281600A3F022AFF0FEE0FCA3E0F5828C83E49304
:10282600FD2275F00EA42401F9743A35F0FA7BFF07
:1028360022EBF0AC07A2AFE433A3F0C2AF22E475FB
:10284600F001020F48EDFFAD04EDCFF0A3EFF0E489
:01285600225F
:06337700E490038CF0223B
:0733640090038C7401F022BC
:102676009003427403F0E4A3F01233557E3A7F00D0
:102686007A037942122724122FB7E4900341F0907F
:102696000341E0FFC394045050745A2FF8767F74B8
:1026A6005E2FF8767F74622FF8E4F6855858E55960
:1026B600549FF559FFE55854FEF558EF547FF559E8
:1026C600FFE55854F9F5588F5954E7F5588F59F5E1
:1026D60058EF54FCF55985585854FBF55985585808
:1026E60054E7F559E004F080A6E4900341F0900326
:1026F60041E0FFC3941E501575F00EEF1227DD1250
:1027060027F9122E79900341E004F080E1122FB7E9
:0E2716007E3B7FA57A037943122724022FB75A
:0E2724007B01900367E4F0A304F0122E7922EB
:10310E00302011202D1630241390038CE07002D243
:0D311E0025D22D22202805D2281225B2220C
:1031E600903BA5E493F46009903A00E4936403608D
:0A31F60003122676E490037DF02218
:1030AE0090037DE0FFC3941E5016EF122828785827
:1030BE007C007D007E007F0E120E2BC22D1225B2DB
:0130CE0022DF
:1031470090037DE0C3941E501212335590037D12F5
:0C31570027D91227F9122E79122FB72267
:06337D00123147C22D22AF
:0528570090035BEDF0B1
:10285C0090035DE004F0900360EFF0A3EBF09003C5
:10286C005BE0FF900360E0FED39F505E75F00EEED0
:10287C001227DD900362EEF0A3EFF09003611227B4
:10288C00D9900364EEF0A3EFF0E490035EF0A3F0B4
:10289C009003641228449003621228191229D290D2
:1028AC0003621227F290035E1227F2C390035FE0DB
:1028BC00940E90035EE0940040D6122FB790036004
:0A28CC00E004F0A3E004F002286A23
:0128D60022DF
:0524E50090035AEDF028
:1024EA0090035FEFF0A3EBF090035AE0FF90035FD5
:1024FA00E0D39F40030225B1A31227D912280990DD
:10250A000361E0FEA3E0FFC3940EEE9400501A901C
:10251A00035B12281C747E2FF582E43403F583EDE5
:10252A00F090035B1227E880D61227D690035DEE5F
:10253A00F0A3EFF09003601227D912280990035BE9
:10254A0012284490035D1228191229D290035D12B1
:10255A0027E8C3900362E0940E900361E094004080
:10256A00DC1227D690035D12280C900361E0FCA3CD
:10257A00E0FDC3940EEC9400501D90035D122844B4
:10258A00AFF0FE747E2DF582E43403F583E0FD128C
:10259A0029D21227EF80D3122FB790035FE004F0FD
:0725AA00A3E004F00224F29B
:0125B1002207
:0329550090035A92
:1029580012283712335D90036012284B90035CF005
:1029680090035AE0FF900360E0FCA3E0FD7B017A4E
:1029780003797E90036812280212308C900360E479
:1029880075F00E120F3290035CE0122828A3121182
:102998006012335590035D121140AE02AF017B0106
:1029A8007A03797E1227FF122E79122FB790035CD3
:1029B800E004F0E0C3941E40A790029BE0FF1232AF
:0929C800DA90035BE024FF92AFFA
:0129D10022E3
:032C0B0090035AD9
:102C0E0012283712335D90035D12284B90035CF04F
:102C1E0090035CE0FFC3941E503D75F00EEF12273B
:102C2E00DD90035FEEF0FAA3EFF0FB90035AE0FFA6
:102C3E0090035DE0FCA3E0FDA9037BFF9003671208
:102C4E0028021231CC90035DE475F00E120F329013
:102C5E00035CE004F080B990029BE0FF1232DA9040
:072C6E00035BE024FF92AFBD
:012C7500223C
:102EE300ED8FF0A4AAF08BF0A42480E5F03400FC6D
:102EF3008AF0EBA42CFFE5F03400FE22ED8FF0A462
:0E2F0300AAF0ED8EF0A42AFFE5F03400FE22C5
:03000000020800F3
:03000300021A03DB
:03000B00021A06D0
:03001300021A09C5
:03001B00021A0CBA
:03002300021A0FAF
:03002B00021A12A4
:03003300021A1599
:03003B00021A188E
:03004300021A1B83
:03004B00021A1E78
:03005300021A216D
:03005B00021A2462
:03006300021A2757
:03006B00021A2A4C
:03007300021A2D41
:10080000E4F5D9E5EF7480F5FF7402F5EF787FE445
:10081000F6D8FD9000007F007E04E4F0A3DFFCDE4C
:07082000FA75816502086210
:100827000211E8E493A3F8E493A34003F68001F2EE
:1008370008DFF48029E493A3F85407240CC8C333D2
:10084700C4540F4420C8834004F456800146F6DFA1
:10085700E4800B0102040810204080902F68E47E9A
:10086700019360BCA3FF543F30E509541FFEE49396
:10087700A360010ECF54C025E060A840B8E493A35D
:10088700FAE493A3F8E493A3C8C582C8CAC583CA88
:10089700F0A3C8C582C8CAC583CADFE9DEE780BE40
:012F90000040
:100D5B00E709F608DFFA8046E709F208DFFA803E7A
:100D6B0088828C83E709F0A3DFFA8032E309F60867
:100D7B00DFFA8078E309F208DFFA807088828C83CF
:100D8B00E309F0A3DFFA806489828A83E0A3F60883
:100D9B00DFFA805889828A83E0A3F208DFFA804C5D
:100DAB0080D280FA80C680D4806980F28033801034
:100DBB0080A680EA809A80A880DA80E280CA80339D
:100DCB0089828A83ECFAE493A3C8C582C8CCC58315
:100DDB00CCF0A3C8C582C8CCC583CCDFE9DEE780E5
:100DEB000D89828A83E493A3F608DFF9ECFAA9F064
:100DFB00EDFB2289828A83ECFAE0A3C8C582C8CCBA
:100E0B00C583CCF0A3C8C582C8CCC583CCDFEADED2
:100E1B00E880DB89828A83E493A3F208DFF980CC34
:100E2B0088F0EF60010E4E60C388F0ED2402B4042D
:100E3B000050B9F582EB2402B4040050AF232345D4
:060E4B008223900DAB7341
:100E5100BB010689828A83E0225002E722BBFE029F
:090E6100E32289828A83E49322D2
:100E6A00BB010CE58229F582E5833AF583E022503D
:100E7A0006E92582F8E622BBFE06E92582F8E22287
:0D0E8A00E58229F582E5833AF583E49322A1
:100E9700BB010689828A83F0225002F722BBFE013A
:020EA700F32234
:100EA900F8BB010DE58229F582E5833AF583E8F07F
:100EB900225006E92582C8F622BBFE05E92582C82B
:020EC900F22213
:100ECB00EF8DF0A4A8F0CF8CF0A428CE8DF0A42E3B
:020EDB00FE22F5
:100EDD00BC000BBE0029EF8DF084FFADF022E4CCF9
:100EED00F875F008EF2FFFEE33FEEC33FCEE9DECC2
:100EFD00984005FCEE9DFE0FD5F0E9E4CEFD22ED08
:100F0D00F8F5F0EE8420D21CFEADF075F008EF2F51
:100F1D00FFED33FD4007985006D5F0F222C398FD42
:050F2D000FD5F0EA22DF
:100F3200C5F0F8A3E028F0C5F0F8E582158270024A
:060F42001583E038F022E7
:100F4800A3F8E0C5F025F0F0E5821582700215835C
:060F5800E0C838F0E822B9
:0D0F5E00EF2BFFEE3AFEED39FDEC38FC22E2
:0E0F6B00C3EF9BFFEE9AFEED99FDEC98FC2281
:100F7900E88FF0A4CC8BF0A42CFCE98EF0A42CFC17
:100F89008AF0EDA42CFCEA8EF0A4CDA8F08BF0A495
:100F99002DCC3825F0FDE98FF0A42CCD35F0FCEBF4
:100FA9008EF0A4FEA9F0EB8FF0A4CFC5F02ECD39B9
:0F0FB900FEE43CFCEAA42DCE35F0FDE43CFC2226
:100FC80075F008758200EF2FFFEE33FECD33CDCCE0
:100FD80033CCC58233C5829BED9AEC99E582984063
:100FE8000CF582EE9BFEED9AFDEC99FC0FD5F0D640
:100FF800E4CEFBE4CDFAE4CCF9A88222B800C1B96A
:101008000059BA002DEC8BF084CFCECDFCE5F0CBA7
:10101800F97818EF2FFFEE33FEED33FDEC33FCEBE0
:1010280033FB10D703994004EB99FB0FD8E5E4F99B
:10103800FA227818EF2FFFEE33FEED33FDEC33FC88
:10104800C933C910D7059BE99A4007EC9BFCE99A7C
:10105800F90FD8E0E4C9FAE4CCFB2275F010EF2FC1
:10106800FFEE33FEED33FDCC33CCC833C810D707C1
:101078009BEC9AE899400AED9BFDEC9AFCE899F8FC
:0E1088000FD5F0DAE4CDFBE4CCFAE4C8F9228F
:102D7B00C2D5E830E70FB2D5E4C39BFBE49AFAE483
:102D8B0099F9E498F8EC30E717B2D5122DB112107F
:102D9B0004E4C39BFBE49AFAE499F9E498F8800302
:102DAB0012100430D50DE4C39FFFE49EFEE49DFD9D
:042DBB00E49CFC2276
:10109600EB9FF5F0EA9E42F0E99D42F0EC6480C8D1
:0610A60064809845F02271
:1010AC00E8600FECC313FCED13FDEE13FEEF13FF22
:0310BC00D8F12246
:0C10BF00E0FCA3E0FDA3E0FEA3E0FF22A4
:0C10CB00E0F8A3E0F9A3E0FAA3E0FB22A8
:1010D7007401FF3395E0FEFDFC080808E6CF2FF604
:1010E70018E6CE3EF618E6CD3DF618E6CC3CF622DD
:0C10F700ECF0A3EDF0A3EEF0A3EFF0226C
:10110300A8828583F0D083D08212111A12111A1289
:10111300111A12111AE473E493A3C583C5F0C583AE
:10112300C8C582C8F0A3C583C5F0C583C8C582C836
:011133002299
:0C113400A42582F582E5F03583F58322C6
:09114000E0FBA3E0FAA3E0F922B0
:10114900F8E0FBA3A3E0F925F0F0E582158270022F
:071159001583E0FA38F022D3
:09116000EBF0A3EAF0A3E9F02290
:10116900D083D082F8E4937012740193700DA3A315
:1011790093F8740193F5828883E473740293686029
:06118900EFA3A3A380DF29
:10118F00EC8EF0A4CCC5F0CCCDF8EFA4CEC5F02DED
:10119F00FDE43CFCE8A42EC8C5F03DFDE43CFCEFAB
:0D11AF00A4FFE5F028FEE43DFDE43CFC2239
:1011BC00EF4E6012EF60010EEDBB010B89828A834A
:1011CC00F0A3DFFCDEFA2289F05007F709DFFCA957
:0C11DC00F022BBFEFCF309DFFCA9F022AE
:00000001FF
